:021DFE00820061
:101E0000003401340234023403340434053406341B
:101E100006340734083409340A340A340B340C34D9
:101E20000D340E340F340F34103411341234133493
:101E300014341534153416341734183419341A344C
:101E40001B341C341D341E341E341F342034213402
:101E500022342334243425342634273428342834B7
:101E600029342A342B342C342D342E342F3430346E
:101E70003134313432343334343435343634373425
:101E8000383439343A343B343C343D343E343F34D6
:101E90004034413442344334443445344634473486
:101EA000483449344A344B344C344D344E344F3436
:101EB00050345134523453345434553455345634E8
:101EC0005734583459345A345B345C345D345E349E
:101ED0005F3460346134623463346534663467344B
:101EE000683469346A346B346C346D346E346F34F6
:101EF000713472347334743475347634773478349E
:101F00007A347B347C347D347E3480348134823442
:101F10008334843485348734883489348A348C34E7
:101F20008D348E348F349134923493349534963486
:101F3000973499349A349B349D349E34A034A13420
:101F4000A234A434A534A734A834A934AB34AC34B7
:101F5000AE34AF34B034B234B334B534B634B8344C
:101F6000B934BB34BC34BE34BF34C134C234C434DD
:101F7000C534C734C834CA34CB34CD34CF34D0346C
:101F8000D234D434D534D734D934DA34DC34DE34F2
:101F9000E034E134E334E534E734E834EA34EC3473
:101FA000EE34F034F234F434F634F834FB34FD34E7
:101FB000FF34FF34FF34FF34FF34FF34FF34FF3489
:101FC000FF34FF34FF34FF34FF34FF34FF34FF3479
:101FD000FF34FF34FF34FF34FF34FF34FF34FF3469
:101FE000FF34FF34FF34FF34FF34FF34FF34FF3459
:101FF000FF34FF34FF34FF34FF34FF34FF34FF3449
:00000001FF
